:03000000020006F5
:1E005F007508807509C3750AC9750B01751B01751C00751D00751E00751F000200039C
:03000300023FB702
:20007D007F06DFFE227F26DFFE227F4EDFFE22007F8C7E02DFFEDEFC227F1B7E04DFFEDE34
:20009D00FC22007F287E20DFFEDEFC22AE82AF83C3EE9401EF940050047E017F00C007C003
:2000BD000612009FD006D0071EBEFF011FEE4F70EC22AF82C00712007DD007DFF7224391DF
:2000DD0020439220439110439210D294D29522439110439210D294D2957582041200CFC202
:2000FD00947582041200CFC29522439110439210C295C2947582041200CFD2957582011237
:20011D0000CFD2947582040200CF439110AF9274EF5FF592D2947582011200CFD2957582B6
:20013D00011200CF7F0030940D0FEF240550F712010775820122C29575820022C295439133
:20015D0010439210C2947582021200CFD2957582021200CFC29522C295439110439210D2B1
:20017D00947582021200CFD2957582021200CFC29522AF82439110439210C2957E00748077
:20019D005F23540124FF9294EF2FFF758202C007C0061200CFD2957582021200CFC2957591
:2001BD0082021200CFD006D0070EBE080040CF227F00439110AE9274EF5EF5927E00C2954B
:2001DD00758202C007C0061200CFD006D007D295EF2FFF3094010F758201C007C0061200FF
:2001FD00CFD006D0070EBE080040D38F8222C02E85812EAF82C0071200ECD0078F82C00785
:20021D0012018F120127E52E24FDF8868212018F1201271200ECD00774014FF58212018F23
:20023D00120127E52E24F9F88607E52E24FAF88604088605088606C007C006C005C00412B0
:20025D0001CDAB82D004D005D006D0078C828D838EF0EB123FBFA3AC82AD83BF0102801343
:20027D00C007C006C005C004120159D004D005D006D007DFC2120174120107D02E22C02E39
:20029D0085812EAF82C0071200ECD0078F8212018F120127E52E24FDF8868212018F12016A
:2002BD0027E52E24FAF88605088606088607E52E24F9F886048D828E838FF01241E5FBA3F6
:2002DD00AD82AE838B82C007C006C005C00412018F120127D004D005D006D007DCD7120186
:2002FD0007D02E220200DBC02E85812EAE82AF83C007C0061200ECD006D0078F04EC2C2452
:20031D00A0F582C007C00612018F120127D006D0078E8212018F120127E52E24FDF8868273
:20033D0012018F120127120107D02E22AE82AF83C007C0061200ECD006D0078F04EC2C2421
:20035D00A0F582C007C00612018F120127D006D0078E8212018F1201271200EC7582A112BF
:20037D00018F1201271201CDAF82C007120174120107D0078F8222C02E85812EC082C0836C
:20039D007D00E52E24F9F8C3ED965052ED75F008A4FB8BF005F0E52E24FAF8860308860208
:2003BD00088604088607800DC3EF13FFEC13FCEA13FAEB13FBD5F0F08D067F00A82E08EE2A
:2003DD0026FEEF0836FFC005C0038E828F8312030415819000051200A9D0050D80A4852E4E
:2003FD0081D02E22C02E85812EC082C083E5812404F581E52E2403F8E4F608F608F608F68E
:20041D007F00E52E24FDF8C3EF965063E52E2403F80808E608F61818E608F61818E608F6CB
:20043D00187600E52E24FDF886057E00A82E08ED26FDEE0836FE8F037C00EDC39BFDEE9CE4
:20045D00FEED24FFF582EE34FFF583C007120349AE82D007E4FDFCFBE52E2403F8EE26F621
:20047D00ED0836F6EC0836F6EB0836F60F8093E52E2403F886820886830886F008E6852E73
:20049D0081D02E22C02E85812E0581AE82AF83E52E24FBF88603088604088605A82E087668
:2004BD0000C006C007A82E0886067F00E52E24F9F8C3EE96EF0896D007D006503F8B828CD8
:2004DD00838DF01241E5FAA3AB82AC83C007C006C005C004C003C0028E828F8312030415E3
:2004FD00819000051200A9D003D004D005D006D0070EBE00010FA82E080680A51581D02E6C
:20051D0022C02E85812E0581AE82AF83E52E24FBF88603088604088605A82E087600C006A0
:20053D00C007A82E0886067F00E52E24F9F8C3EE96EF0896D007D00650378E828F83C007D5
:20055D00C006C005C004C003120349AA82D003D004D005D006D0078B828C838DF0EA123FE5
:20057D00BFA3AB82AC830EBE00010FA82E080680AD1581D02E22AF82AE9574DF5EF595AEA0
:20059D009674DF5EF596AE9574EF5EF595AE9674EF5EF596AE9574F75EF595AE9674F75EAB
:2005BD00F59643CE8043CE40AECE74DF5EF5CE43CE10AECE74F75EF5CE85CECEAECE74FB8C
:2005DD005EF5CE85CECEAECE5306FCEF4EF5CEAFA274F35F4404F5A2C2A5D2A375CDC022F5
:2005FD008582CFE5CD30E7FB75CDC02275CFFFE5CD30E7FB75CDC085CF82228582CFE5CD97
:20061D0030E7FB75CDC085CF8222C2C822D2C8220205FDAE82AF838F82C007C00612062D00
:20063D00D006D0078E8202062DAF82C2B78F8212062DD2B722758200120593AFC974FD5F17
:20065D00F5C943CA02AFC974FE5FF5C943CA01AFB1747F5FF5B143B280C2A522D2C990001A
:20067D00321200A9C2C99000641200A9D2C99000320200A9C02E85812EAE82AF83E512FDB6
:20069D00705D75822AC007C006120646D006D007E5132EF582E5143FF583120630E52E24EB
:2006BD00FAF8E51326F582E5140836F58312063075822B120646E52E24FCF8E51726F5825B
:2006DD00E5180836F583120630E52E24F8F8E51726F582E5180836F58312063002081CBD64
:2006FD00015D75822AC007C006120646D006D007E5172EF582E5183FF583120630E52E24F2
:20071D00FAF8E51726F582E5180836F58312063075822B120646E52E24FCF8E51526F582F4
:20073D00E5160836F583120630E52E24F8F8E51526F582E5160836F58312063002081CBD09
:20075D00025C75822AC007C006120646D006D007E5152EF582E5163FF583120630E52E2495
:20077D00FAF8E51526F582E5160836F58312063075822B120646E52E24FCF8E51926F58294
:20079D00E51A0836F583120630E52E24F8F8E51926F582E51A0836F5831206308061BD03DF
:2007BD005C75822AC007C006120646D006D007E5192EF582E51A3FF583120630E52E24FA35
:2007DD00F8E51926F582E51A0836F58312063075822B120646E52E24FCF8E51326F582E547
:2007FD00140836F583120630E52E24F8F8E51326F582E5140836F58312063080028006759A
:20081D00822C120646D02E22C02E85812EAE82AF83E52E24FCF8E6C0E008E6C0E0C006C046
:20083D0007E52E24FCF8E6C0E008E6C0E08E828F83120691E58124FAF581D02E22C02E85FD
:20085D00812EAE82AF838E0C8F0DE52E24FCF8860E08860FAE0CAF0DBE502BBF002874A02E
:20087D00B50E06E4B50F028002801B75131A75140075151A751600751701751800751901C8
:20089D00751A00020913E4BE8004BF000104FD60217480B50E06E4B50F0280028014E4F5D0
:2008BD0013F514F515F516F517F518751920F51A8044ED602074A0B50E06E4B50F028002DA
:2008DD008013E4F513F514F515F516F517F518F519F51A8021BEF01EBF001B7440B50E1654
:2008FD007401B50F11E4F513F514F515F516F517F518F519F51A12065212067912062775A2
:20091D0082111206469000321200A975823612064675820012062D9000321200A975823AD7
:20093D0012064675820512062D7582B212064675820C12062D75820C12062D758200120655
:20095D002D75823312062D75823312062D7582B712064675823512062D7582BB120646756D
:20097D00823512062D7582C012064675822C12062D7582C212064675820112062D7582C3D3
:20099D0012064675821312062D7582C412064675822012062D7582C612064675820F1206DF
:2009BD002D7582CA12064675820F12062D7582C812064675820812062D7582551206467503
:2009DD00829012062D7582D01206467582A412062D7582A112062D7582E01206467582D0C5
:2009FD0012062D75820012062D75820612062D75820912062D75820B12062D75822A120652
:200A1D002D75823C12062D75825512062D75824B12062D75820812062D75821612062D75F1
:200A3D00821412062D75821912062D75822012062D7582E11206467582D012062D758200D4
:200A5D0012062D75820612062D75820912062D75820B12062D75822912062D7582361206BC
:200A7D002D75825412062D75824B12062D75820D12062D75821612062D75821412062D75B5
:200A9D00822112062D75822012062D758229120646D02E22C02E85812EAE82AF838E138FA3
:200ABD0014E52E24FCF88615088616E52E24FAF88617088618E52E24F8F8861908861AD0F1
:200ADD002E22C02E85812EAF82C007120627758236120646D007EF035480FFE52E24FDF8FD
:200AFD00E6030354C04207E52E24FCF8E6C42354E04207E52E24FBF8E6C454F04207E52EA7
:200B1D0024F9F8E625E025E042078F8212062D12062AD02E22AF82AE9174F75EF59143921E
:200B3D0008EF7003C29322D29322AF828F12120627E512FF24FC5003020BD9EF2F2F900BE8
:200B5D005F73020B6B020B89020BA3020BC1AE0CAF0D8E0C8F0DAE0EAF0F8E0E8F0F7582C3
:200B7D003612064675820012062D8050AE0EAF0F8E0C8F0D8E0E8F0F75823612064675824C
:200B9D006012062D8036AE0CAF0D8E0C8F0DAE0EAF0F8E0E8F0F7582361206467582C01229
:200BBD00062D8018AE0EAF0F8E0C8F0D8E0E8F0F7582361206467582A012062D02062AC00A
:200BDD002E85812E05810581AE82AF83C007C006120627E50E24FFFCE50F34FFFDE50C2411
:200BFD00FFFAE50D34FFFBC004C005C002C003E4C0E0C0E0900000120691E58124FAF5815A
:200C1D00D006D0078F05A82E08E4F608F6C005AA0CAD0DA82E08C3E69A08E69DD005505565
:200C3D007A007C00C005AB0EAD0FC3EA9BEC9DD00550378D82C007C006C005C004C0021241
:200C5D00062DD002D004D005D0068E038B82C006C005C004C00212062DD002D004D005D0B4
:200C7D0006D0070ABA00BD0C80BAA82E0806B600020806809812062A852E81D02E22C02E6D
:200C9D0085812EAE82AF83C007C006120627D006D007E52E24FCF8E6C0E008E6C0E0C00623
:200CBD00C007E52E24FCF8E6C0E008E6C0E08E828F83120691E58124FAF581E52E24FAF823
:200CDD0008868212062DE52E24FAF886078F8212062D12062AD02E22C02E85812EC082C010
:200CFD0083E581240EF581E52E240EF8E4F608F6087600E52E24FBF88602E52E24FBF8EAED
:200D1D0024E0F6E52E24F6F8B60C28E52E240DF87608E52E24FBF8E675F00CA424F0FE7448
:200D3D005135F0FFE52E240EF8A60608A6070876808055E52E24F6F8B61009E52E240DF880
:200D5D0076088044E52E24F6F8B61809E52E240DF876108033E52E24F6F8B62028E52E2469
:200D7D000DF87610E52E24FBF8E675F040A42464FE745635F0FFE52E240EF8A60608A60760
:200D9D000876808003021416A82E0808E620E7030210A3E52E240AF87600E52E240AF8E531
:200DBD002E24F6F9C3E6974003021416E52E240AF8E52E240DF986F0E7A4FCADF0E52E24DF
:200DDD0005F8A60408A605E52E24F6F8E6C313FBE52E2409F87600E52E2409F8C3E69B4056
:200DFD000302109AC004C005E52E2409F8E52E2407F9E6F7097700A82E08E52E2407F9E7D6
:200E1D002609E70836D005D00430E703021091C004C005A82E08E52E2407F9E726FC09E764
:200E3D000836FD8B027F00ECC39AFCED9FFDC3E50C9CE50D64808DF063F08095F0D005D0E0
:200E5D00045003021416E52E24F6F886067F00E52E24FCF8EE26FEEF0836FFC3E50E9EE520
:200E7D000F64808FF063F08095F05003021416E52E24F5F8E66003020FBCC003E52E2407D1
:200E9D00F8E62CFE08E63DFFE52E240BF8A60608A607E52E240BF8860208E6C423CAC42320
:200EBD00541F6ACA541FCA6ACAFBE52E240EF8EA26FAEB0836FB0886078A828B838FF01257
:200EDD0041E5FAE52E240BF8740756FE8EF005F07E017F008006EE2EFEEF33FFD5F0F77B63
:200EFD0000EE5202EF5203EA4BD0036059C004C005E52E240AF886027F00E52E24FCF8EAB0
:200F1D0026FAEF0836FFA82E08E52E2407F9E726FD09E70836FEC005C004C003E52E24F9A1
:200F3D00F8E6C0E008E6C0E0C002C0078D828E83120C9BE58124FCF581D003D004D005D0DE
:200F5D0005D004021091C004C005E52E240AF886027F00E52E24FCF8EA26FAEF0836FFA826
:200F7D002E08E52E2407F9E726FD09E70836FEC005C004C003E52E24F7F8E6C0E008E6C00B
:200F9D00E0C002C0078D828E83120C9BE58124FCF581D003D004D005D005D004021091C06E
:200FBD0004C005E52E2405F8E52E2407F9E726FE09E70836FFE52E240BF8A60608A607E528
:200FDD002E240BF8860608E6C423CEC423541F6ECE541FCE6ECEFFE52E240EF8EE26FEEF20
:200FFD000836FF0886028E828F838AF01241E5FEE52E240BF8740756FA8AF005F07A017FC7
:20101D00008006EA2AFAEF33FFD5F0F78E057E00EA5205EF5206ED4ED005D0046056C0044B
:20103D00C005E52E240AF886027F00E52E24FCF8EA26FAEF0836FFA82E08E52E2407F9E731
:20105D0026FD09E70836FEC005C004C003E52E24F9F8E6C0E008E6C0E0C002C0078D828E76
:20107D0083120C9BE58124FCF581D003D004D005D005D004E52E2409F806020DF4E52E247E
:20109D000AF806020DB7E52E240AF87600E52E240AF8E52E24F6F9C3E6974003021416E5C3
:2010BD002E240AF8E52E240DF986F0E7A4FDAEF08D038E04E52E24F6F8E6C313FAE52E24B2
:2010DD0009F87600E52E2409F8C3E69A400302140DC003C004E52E2409F8E52E2407F9E6BF
:2010FD00F7097700A82E08E52E2407F9E726C0E009E70836C0E0E52E2406F8D0E0F618D009
:20111D00E0F68A047F00E52E2405F8E6C39CFC08E69FFFC3E50C9CE50D64808FF063F08056
:20113D0095F0D004D0035003021416C003C004E52E24F6F886047F00E52E24FCF8EC26FCF9
:20115D00EF0836FFC3E50E9CE50F64808FF063F08095F0D004D0035003021416E52E24F5F3
:20117D00F8E660030212FDC003C004E52E2407F8E62DFC08E63EFFE52E240BF8A60408A677
:20119D0007E52E240BF8860408E6C423CCC423541F6CCC541FCC6CCCFFE52E240EF8EC266F
:2011BD00FCEF0836FF0886038C828F838BF01241E5FCE52E240BF8740756FB7F008BF00585
:2011DD00F0E52E2405F87601087600188009E625E0F608E633F618D5F0F4E52E2403F8A697
:2011FD0004087600E52E2405F88603088607E52E2403F8E6520308E65207EB4FD004D00369
:20121D00606FC003C004E52E240AF886047F00E52E24FCF8E52E2403F9EC26F7EF0836097C
:20123D00F7A82E08E52E2407F9E726FB09E70836FFC006C005C004C003C002E52E24F9F854
:20125D00E6C0E008E6C0E0E52E2403F8E6C0E008E6C0E08B828F83120C9BE58124FCF58143
:20127D00D002D003D004D005D006D004D003021404C003C004E52E240AF886047F00E52E90
:20129D0024FCF8E52E2403F9EC26F7EF083609F7A82E08E52E2407F9E726FB09E70836FF66
:2012BD00C006C005C004C003C002E52E24F7F8E6C0E008E6C0E0E52E2403F8E6C0E008E65D
:2012DD00C0E08B828F83120C9BE58124FCF581D002D003D004D005D006D004D00302140498
:2012FD00C005C006E52E2407F8E62BFE08E63CFFE52E240BF8A60608A607E52E240BF8867D
:20131D000608E6C423CEC423541F6ECE541FCE6ECEFFE52E240EF8EE26FEEF0836FF0886EC
:20133D00058E828F838DF01241E5FEE52E240BF8740756FD7F008DF005F0E52E2403F87615
:20135D0001087600188009E625E0F608E633F618D5F0F4E52E2405F8A606087600E52E24F2
:20137D0003F88605088607E52E2405F8E6520508E65207ED4FD006D005606CC003C004E55E
:20139D002E240AF886047F00E52E24FCF8E52E2403F9EC26F7EF083609F7A82E08E52E242A
:2013BD0007F9E726FB09E70836FFC006C005C004C003C002E52E24F9F8E6C0E008E6C0E0CB
:2013DD00E52E2403F8E6C0E008E6C0E08B828F83120C9BE58124FCF581D002D003D004D08D
:2013FD0005D006D004D003E52E2409F8060210E1E52E240AF8060210AA852E81D02E22C00E
:20141D002E85812EC082C083E52E24F4F8E6C313FDE52E24F9F886020886030886048A820D
:20143D008B838CF01241E5FF24814072BF2000406DC005C004C003C002E52E24F3F8E6C015
:20145D00E0E52E24F4F8E6C0E0E52E24F5F8E6C0E008E6C0E0E52E24F7F8E6C0E008E6C054
:20147D00E0C007E52E24FCF8E6C0E008E6C0E0A82E088682088683120CF5E58124F7F58168
:20149D00D002D003D004D0058D067F00A82E08EE26F6EF0836F60ABA00010B02143B852EF0
:2014BD0081D02E22C02E85812EC082E5812414F581120627E52E24F9F808E620E70302187D
:2014DD004BE52E24F9F8C3E496FD08E496FE740CC0E0E4C0E08D828E83124246AD82AE8304
:2014FD0015811581A82E08C3ED964003021B66ED75F018A4FCAEF08C028E03E52E240EF8B5
:20151D00ED75F00CA4F608A6F0E52E240EF8E52E24F9F9E726C0E009E70836C0E0E52E2400
:20153D0013F8D0E0F618D0E0F6E52E2412F8E52E240CF9E6F70809E6F7E52E2412F8E52E83
:20155D002408F9E6F70809E6F7E52E2412F8E52E2410F9E6F70809E6F7E52E2415F8760078
:20157D00C005E52E2415F8E675F002A4FDAFF0A82E0808ED2CF6EF3E08F6E52E2404F8ED78
:20159D002AF6EF3B08F6E52E2414F87600D005C002C003E52E2414F8E52E2406F9E6F70974
:2015BD007700E52E240EF8E52E2406F9E726FB09E70836FFE52E24F9F8E62BFB08E63FFF8F
:2015DD00EB24F4FBEF34FFFFC374EF9B74808FF063F08095F0D003D0025003021B69C00203
:2015FD00C003E52E2415F8E52E240AF9E6F7097700E52E24F7F8E52E240AF9E726FB09E7D8
:20161D000836FFEB24F4FBEF34FFFFC374539B74818FF063F08095F0D003D0025003021B4B
:20163D0069C002C003E52E2410F8E52E2406F9E72609E70836FFD003D00230E703021821F6
:20165D00E52E24F2F8E66003021774C002C003E52E2414F8E6C423541FFB7F00A82E08080E
:20167D00EB26FBEF0836FFE52E24FBF8EB26FBEF0836FF0886028B828F838AF01241E5FB57
:20169D00E52E2414F8740756F5F005F074808002C313D5F0FBFF5BD003D002605DC002C0F5
:2016BD0003E52E24F7F8E52E240AF9E726FB09E70836FFE52E2408F8E52E2406F9E726F506
:2016DD008209E70836F583C006C005C004C003C002C003C00712082515811581E52E24F5D0
:2016FD00F88682088683120630D002D003D004D005D006D003D002021821C002C003E52ED8
:20171D0024F7F8E52E240AF9E726FB09E70836FFE52E240CF8E52E2406F9E726F58209E745
:20173D000836F583C006C005C004C003C002C003C00712082515811581E52E24F3F88682E3
:20175D00088683120630D002D003D004D005D006D003D002021821C002C003E52E2414F847
:20177D00E6C423541FFB7F00E52E2404F8EB26FBEF0836FFE52E24FBF8EB26FBEF0836FFC5
:20179D000886028B828F838AF01241E5FBE52E2414F8740756F5F005F074808002C313D5C1
:2017BD00F0FBFF5BD003D002605AC002C003E52E24F7F8E52E240AF9E726FB09E70836FF4E
:2017DD00E52E2412F8E52E2406F9E726F58209E70836F583C006C005C004C003C002C003B4
:2017FD00C00712082515811581E52E24F5F88682088683120630D002D003D004D005D006F1
:20181D00D003D002E52E2414F806E52E2414F8B60C0050030215ACE52E2415F806E52E2421
:20183D0015F8B60C00500302157D0D0215017F00A82E08C3EF964003021B66EF75F018A435
:20185D00FDAEF08D038E04E52E240AF8EF75F00CA4F608A6F0E52E240AF8E52E24F9F9E794
:20187D0026C0E009E70836C0E0E52E2407F8D0E0F618D0E0F6E52E2406F8E52E2404F9E6CE
:20189D00F70809E6F7E52E2406F8A92E0909E6F70809E6F7E52E2415F87600C007E52E24A5
:2018BD0015F8E675F002A4FAAFF0E52E2410F8EA2DF6EF3E08F6E52E2408F8EA2BF6EF3C90
:2018DD0008F6E52E2414F87600D007C003C004E52E2414F8E52E240CF9E6F7097700E52EE7
:2018FD00240AF8E52E240CF9E726FA09E70836FCE52E24F9F8E62AFA08E63CFCEA24F4FAE4
:20191D00EC34FFFCC374EF9A74808CF063F08095F0D004D0035003021B69C003C004E52EED
:20193D002415F8E52E2412F9E6F7097700E52E24F7F8E52E2412F9E726FA09E70836FCEA37
:20195D0024F4FAEC34FFFCC374539A74818CF063F08095F0D004D0035003021B69E52E2499
:20197D00F2F8E66003021A90C003C004E52E2414F8E6C423541FFA7C00E52E2410F8EA269C
:20199D00FAEC0836FCE52E24FBF8EA26FAEC0836FC0886038A828C838BF01241E5FAE52E44
:2019BD002414F8740756F5F005F074808002C313D5F0FB5AD004D003605CC003C004E52ECC
:2019DD0024F7F8E52E2412F9E726FA09E70836FCA82E0808E52E240CF9E726F58209E708C6
:2019FD0036F583C007C006C005C004C003C002C00412082515811581E52E24F5F88682081E
:201A1D008683120630D003D004D005D006D007D004D003021B3CC003C004E52E24F7F8E59D
:201A3D002E2412F9E726FA09E70836FCE52E2404F8E52E240CF9E726F58209E70836F58362
:201A5D00C007C006C005C004C003C002C00412082515811581E52E24F3F886820886831252
:201A7D000630D003D004D005D006D007D004D003021B3CC003C004E52E2414F8E6C42354FF
:201A9D001FFA7C00E52E2408F8EA26FAEC0836FCE52E24FBF8EA26FAEC0836FC0886038AB8
:201ABD00828C838BF01241E5FAE52E2414F8740756F5F005F074808002C313D5F0FB5AD0A7
:201ADD0004D003605AC003C004E52E24F7F8E52E2412F9E726FA09E70836FCE52E2406F803
:201AFD00E52E240CF9E726F58209E70836F583C007C006C005C004C003C002C004120825C5
:201B1D0015811581E52E24F5F88682088683120630D003D004D005D006D007D004D003E542
:201B3D002E2414F806E52E2414F8B60C0050030218E8E52E2415F806E52E2415F8B60C007A
:201B5D0050030218B80F02184D12062A852E81D02E22C02E85812EC082E5812419F58112A8
:201B7D000627E52E24F9F808E620E703021ECEE52E24F9F8C3E496FD08E496FE7420C0E0F7
:201B9D00E4C0E08D828E83124246AD82AE8315811581A82E08C3ED964003022255E52E2447
:201BBD0011F8ED75F080A4F608A6F0ED75F020A4FAABF0E52E24F9F8E62AFA08E63BFBE50F
:201BDD002E2411F8E52E2407F9E6F70809E6F7E52E2409F8A60208A603A82E0808A6020864
:201BFD00A603E52E2404F8ED75F022A4F608A6F0E52E2404F8E52E24F9F9E726C0E009E747
:201C1D000836C0E0E52E2414F8D0E0F618D0E0F6E52E2419F87600E52E2419F8E52E240BDA
:201C3D00F9E6C423541FF7E52E2419F8740756F5F005F0C8E52E2406C874808002C313D576
:201C5D00F0FBF6E52E240BF8E52E2415F9E6F7E52E2406F8E52E240CF9E6F7E52E2418F895
:201C7D007600C005E52E2418F8E52E240DF9E6F7097700E52E2404F8E52E240DF9E726FDB1
:201C9D0009E70836FFE52E24F9F8E62DFD08E63FFFED24DEFDEF34FFFFC3742B9D74818F06
:201CBD00F063F08095F0D0055003022258C005E52E2419F8E52E240FF9E6F7097700E52E5F
:201CDD0024F7F8E52E240FF9E726FD09E70836FFED24DEFDEF34FFFFC3748F9D74818FF07A
:201CFD0063F08095F0D0055003022258C005E52E2413F8E52E240DF9E72609E70836FFD07D
:201D1D000530E703021EA4E52E24F2F8E66003021E14C005E52E2418F8E675F004A4C8E579
:201D3D002E2411C826FE08E635F0FCE52E240BF886057F00ED2EFDEF3CFFE52E24FBF8ED8B
:201D5D0026FDEF0836FE0886078D828E838FF01241E5FDE52E2406F8E65DD005604CE52EA3
:201D7D0024F7F8E52E240FF9E726FE09E70836FFA82E0808E52E240DF9E726F58209E7081D
:201D9D0036F583C005C003C002C006C00712082515811581E52E24F5F886820886831206E1
:201DBD0030D002D003D005021EA4E52E24F7F8E52E240FF9E726FE09E70836FFE52E2409BB
:201DDD00F8E52E240DF9E726F58209E70836F583C005C003C002C006C007120825158115C6
:201DFD0081E52E24F3F88682088683120630D002D003D005021EA4C005E52E2418F8E6751D
:201E1D00F004A4C8E52E2407C826FE08E635F0FFE52E2415F886047D00EC2EFEED3FFFE596
:201E3D002E24FBF8EE26FEEF0836FF0886058E828F838DF01241E5FEE52E240CF8E65ED04B
:201E5D00056044E52E24F7F8E52E240FF9E726FE09E70836FFE52E240DF8E62AF58208E66E
:201E7D003BF583C005C003C002C006C00712082515811581E52E24F5F886820886831206FB
:201E9D0030D002D003D005E52E2418F806E52E2418F8B620005003021C7FE52E2419F806D3
:201EBD00E52E2419F8B620005003021C340D021BAFE52E24F7F8E52E2411F9741F26F7E46E
:201EDD00083609F7E52E241AF87600E52E241AF8A92E09C3E6974003022255E52E241AF87A
:201EFD00E675F020A4FBACF0E52E24F9F8EB26FAEC0836FD741F2AFEE43DFFC004C003E57E
:201F1D002E2411F8E6C0E008E6C0E0C006C007E52E24F7F8E6C0E008E6C0E08A828D831240
:201F3D000691E58124FAF581D003D004E52E241AF8E675F080A4FEAFF0E52E2413F8A60609
:201F5D0008A607E52E2416F8A60308A604E52E24F9F8E62BFB08E63CFCE52E240FF8A603CE
:201F7D0008A604E52E240DF8A60308A604E52E2419F87600E52E2419F8E6C423541FFAE5D6
:201F9D002E2419F8740756F5F005F0C8E52E240CC874808002C313D5F0FBF6E52E2415F8FD
:201FBD00A602E52E240CF8E52E2406F9E6F7E52E2418F87600C006C007E52E2418F8E52E6A
:201FDD002404F9E6F7097700E52E2416F8E52E2404F9E726FE09E70836FFE52E24F9F8E6A7
:201FFD002EFE08E63FFFEE24E0FEEF34FFFFC3742B9E74818FF063F08095F0D007D0065092
:20201D0003022258C006C007E52E2419F8A92E0909E6F7097700E52E24F7F8A92E0909E713
:20203D0026FE09E70836FFEE24E0FEEF34FFFFC3748F9E74818FF063F08095F0D007D00644
:20205D005003022258E52E24F2F8E66003022176C003C004E52E2418F8E675F004A4C8E523
:20207D002E2409C82EF6EF35F008F68A047D00E52E2409F8EC26FCED0836FDE52E24FBF847
:20209D00EC26FCED0836FD0886038C828D838BF01241E5FCE52E240CF8E65CD004D003600B
:2020BD005CC006C007E52E24F7F8A92E0909E726FD09E70836FFE52E240DF8E52E2404F964
:2020DD00E726F58209E70836F583C007C006C004C003C002C005C00712082515811581E507
:2020FD002E24F5F88682088683120630D002D003D004D006D007D007D006022226C006C080
:20211D0007E52E24F7F8A92E0909E726FD09E70836FFE52E240FF8E52E2404F9E726F5825F
:20213D0009E70836F583C007C006C004C003C002C005C00712082515811581E52E24F3F8ED
:20215D008682088683120630D002D003D004D006D007D007D006022226C006C007E52E2420
:20217D0018F8E675F004A4C8E52E2413C8C9E52E2409C926F708E635F009F7E52E2415F81F
:20219D0086067F00E52E2409F8EE26FEEF0836FFE52E24FBF8EE26FEEF0836FF0886058E18
:2021BD00828F838DF01241E5FEE52E2406F8E65ED007D0066053C006C007E52E24F7F8A986
:2021DD002E0909E726FD09E70836FFE52E2404F8E62BF58208E63CF583C007C006C004C0FD
:2021FD0003C002C005C00712082515811581E52E24F5F88682088683120630D002D003D00C
:20221D0004D006D007D007D006E52E2418F806E52E2418F8B620005003021FD2E52E241943
:20223D00F806E52E2419F8B620005003021F91E52E241AF806021EE812062A852E81D02E95
:20225D0022C02EE581F52E2406F581AE82AF83E52E24F8F8E52E24FCF9E6C397FC08E60940
:20227D0097FD8C828D83C007C006123FDAAC82AD83D006D007E52E24FAF8E6C39EFA08E674
:20229D009FFB8A828B83C007C006C005C004123FDAAA82AB83D004D005D006D007C3EA9C33
:2022BD00EB64808DF063F08095F0E433FC3395E0FD4C603C8E028F03E52E24FCF8860608DC
:2022DD008607E52E24FCF8A60208A603E52E24FAF88602088603E52E24F8F8E52E24FAF93D
:2022FD00E6F70809E6F7E52E24F8F8A60208A603E52E24FAF8C3E69E08E69F503C8E028FCE
:20231D0003E52E24FAF88606088607E52E24FAF8A60208A603E52E24FCF88602088603E5A8
:20233D002E24F8F8E52E24FCF9E6F70809E6F7E52E24F8F8A60208A603C004C005E52E2407
:20235D00FAF8E6C39EFA08E69FFBE52E24F8F8E52E24FCF9E6C397FC08E60997FD8C828DF0
:20237D0083C007C006C003C002123FDAAC82AD83D002D003E52E2405F8A60408A605C00329
:20239D00C0027402C0E0E4C0E08A828B83124246AC82AD8315811581D002D003D006D00734
:2023BD00A82E08A60408A605E52E24FCF8E52E24F8F9C3E69708E60997D005D004500CE5BA
:2023DD002E2403F87601087600800AE52E2403F876FF0876FFE52E24FAF8C3E69E08E69FF3
:2023FD0050030224C9EC4D603DC007C006C005C004C003C002E52E24F6F8E6C0E008E6C0B4
:20241D00E0C006C007E52E24FCF88682088683120C9BE58124FCF581D002D003D004D005EB
:20243D00D006D007803DC007C006C005C004C003C002E52E24F6F8E6C0E008E6C0E0E52E2E
:20245D0024FCF8E6C0E008E6C0E08E828F83120C9BE58124FCF581D002D003D004D005D03E
:20247D0006D007A82E08E52E2405F9E6C397F608E60997F6A82E0808E630E728C004C00501
:20249D00E52E2403F88604088605E52E24FCF8EC26F6ED0836F6A82E08EA26F6EB0836F679
:2024BD00D005D0040EBE00010F0223F2852E81D02E22C02E85812EAE82AF83E52E24FCF860
:2024DD00E52E24FAF9E726FC09E70836FD1CBCFF011DE52E24F8F8E6C0E008E6C0E0C0048D
:2024FD00C005C006C007E52E24FCF8E6C0E008E6C0E08E828F8312225EE58124F8F581D0B2
:20251D002E22C02E85812EAE82AF83E52E24FAF8E62EFC08E63FFD1CBCFF011DE52E24F843
:20253D00F8E6C0E008E6C0E0E52E24FCF8E6C0E008E6C0E0C004C005E52E24FCF8E6C0E0F9
:20255D0008E6C0E08E828F8312225EE58124F8F581D02E22C02E85812EAE82AF83E52E2449
:20257D00F8F8E52E24FCF9E6C397FC08E60997FD8E028F03E52E24FAF8C3EA96EB089650F4
:20259D005B8C828D83C007C006C005C004123FDAAA82AB83D004D005D006D007C007C00627
:2025BD00C005C004E52E24F6F8E6C0E008E6C0E0C002C003E52E24FCF8E6C0E008E6C0E078
:2025DD008E828F831224CFE58124FAF581D004D005D006D0070EBE00970F8094D02E22C001
:2025FD002E85812EC082C083E581240EF581E52E24FAF8E52E2409F97401C396F7E4089620
:20261D0009F7E52E24FAF8E6C0E008E6C0E090FFFE123FE7AA82AB8315811581E52E24FAE4
:20263D00F88607088606E52E240DF8E4F608F6E52E2403F8A60708A606E52E24F7F806B6DB
:20265D0000020806E52E24F9F8E52E2408F9740156F7E52E24F9F8E52E2405F9740256F70B
:20267D00E52E240BF8A60708A606E52E240FF8E4F608F67E017F00E52E240FF8E52E240B0E
:20269D00F9C3E69708E664800987F063F08095F040030229C5E52E2409F808E620E71EE5D7
:2026BD002E240BF816B6FF02081674022AFAE43BFBE52E2409F8EA26F6EB0836F6C002C02A
:2026DD0003E52E240FF806B60002080674022EFEE43FFFE52E2409F8EE26F6EF0836F6E5C2
:2026FD002E240BF8740126FAE40836FBE52E240FF8C3E69A08E664808BF063F08095F0D0C0
:20271D0003D0024003022856E52E2408F8E670030227BDC006C007E52E240BF8860608E64D
:20273D00CE25E0CE33FFE52E24F7F8E62EFE08E63FFFE52E24FCF8E52E240BF9E6C397C0DF
:20275D00E008E60997C0E0E52E2407F8D0E0F618D0E0F6A82E08E52E240FF9E726FC09E79E
:20277D000836FDC007C006C003C002E52E24F5F8E6C0E008E6C0E0C006C007E52E2406F8F5
:20279D00E6C0E008E6C0E08C828D831224CFE58124FAF581D002D003D006D007D007D006EC
:2027BD00E52E2405F8E67003022856C006C007E52E240BF8860408E6CC25E0CC33FDE52ED0
:2027DD0024F7F8E62CFC08E63DFDE52E24FCF8E52E240BF9E6C397C0E008E60997C0E0E53A
:2027FD002E2407F8D0E0F618D0E0F6A82E08E52E240FF9E6C397FE08E60997FFC007C00692
:20281D00C003C002E52E24F5F8E6C0E008E6C0E0C004C005E52E2406F8E6C0E008E6C0E00C
:20283D008E828F831224CFE58124FAF581D002D003D006D007D007D006E52E240BF8E52E0E
:20285D002403F986F0E7B5F00B0886F009E7B5F0030229B2E52E2408F8E67003022909C0B7
:20287D0006C007E52E240DF8860408E6CC25E0CC33FDE52E24F7F8E62CFC08E63DFDE52E7E
:20289D0024FCF8E52E240DF9E6C397C0E008E60997C0E0E52E2407F8D0E0F618D0E0F6A876
:2028BD002E08E52E2403F9E726FE09E70836FFC007C006C003C002E52E24F5F8E6C0E00896
:2028DD00E6C0E0C004C005E52E2406F8E6C0E008E6C0E08E828F831224CFE58124FAF58162
:2028FD00D002D003D006D007D007D006E52E2405F8E670030229A2C006C007E52E240DF899
:20291D00860408E6CC25E0CC33FDE52E24F7F8E62CFC08E63DFDE52E24FCF8E52E240DF991
:20293D00E6C397C0E008E60997C0E0E52E2407F8D0E0F618D0E0F6A82E08E52E2403F9E6DB
:20295D00C397FE08E60997FFC007C006C003C002E52E24F5F8E6C0E008E6C0E0C004C005A2
:20297D00E52E2406F8E6C0E008E6C0E08E828F831224CFE58124FAF581D002D003D006D085
:20299D0007D007D006E52E240BF8E52E2403F9E6F70809E6F7E52E240FF8E52E240DF9E6CD
:2029BD00F70809E6F7022694852E81D02E22C02E85812EC082C083E52E24FBF8E675F002E7
:2029DD00A42401FCE435F0FDE52E24FBF886027B008A068B07E52E24FCF8E6C39EFE08E662
:2029FD009FFFC003C002E52E24F9F8E6C0E008E6C0E0C004C005C006C007A82E0886820857
:202A1D0086831224CFE58124FAF581D002D003E52E24F9F8E6C0E008E6C0E0E4C0E0C0E08C
:202A3D007403C0E0C002C003E52E24FCF8E6C0E008E6C0E0A82E0886820886831225FCE58F
:202A5D008124F7F581852E81D02E22AE82AF83740AC0E07420C0E07400C0E07440C0E08E49
:202A7D00828F83124179E58124FCF58190002075F04022D2E890002D1200A9C2E890002DCD
:202A9D001200A9D2EA90002D1200A9C2EA90002D0200A9E4C0E0744CC0E07473C0E0E4C007
:202ABD00E0C0E004C0E0E4C0E004C0E0E4C0E074C0C0E07451C0E07480C0E075820212143D
:202ADD00C1E58124F4F581AE1F7F008E828F83122A68AD82AE83AFF0E4C0E0740CC0E074FB
:202AFD004CC0E07473C0E0E4C0E0C0E0C005C006C00704C0E0E4C0E090001B12141CE58155
:202B1D0024F5F58122C02E85812EE582FF704EE52E24FDF8E6FE242FF582E43400F583E057
:202B3D00FD7C0074062DFDE43CFCEE2401F582E43400F583E0FE7B00742C2EF582E43BF573
:202B5D008374FFC0E0747FC0E07404C0E0C005C0041229CBE58124FBF581022C68BF014EE9
:202B7D00E52E24FDF8E6FE242FF582E43400F583E0FD7C0074062DFDE43CFCEE2401F5822B
:202B9D00E43400F583E0FE7B00742C2EF582E43BF583749BC0E07493C0E07404C0E0C00520
:202BBD00C0041229CBE58124FBF581022C68BF024CE52E24FDF8E6FE242FF582E43400F5A9
:202BDD0083E0FD7C0074062DFDE43CFCEE2401F582E43400F583E0FE7B00742C2EF582E4A0
:202BFD003BF583747CC0E004C0E07404C0E0C005C0041229CBE58124FBF581804EBF034B54
:202C1D00E52E24FDF8E6FF242FF582E43400F583E0FE7D0074062EFEE43DFDEF2401F58282
:202C3D00E43400F583E0FF7C00742C2FF582E43CF5837430C0E07484C0E07404C0E0C006F4
:202C5D00C0051229CBE58124FBF581D02E22752A007406B52A02801A7412B52A028013746F
:202C7D0021B52A02800C7425B52A0280057426B52A66AE2A7F008E828F83A3122A68AD82DC
:202C9D00AE83AFF0E52A242FF582E43400F583E0FC7B00E52A2401F582E43400F583E0F973
:202CBD007A00E924F3F9EA34FFFAE4C0E0740CC0E074FFC0E0C0E07430C0E07484C0E0C07A
:202CDD0005C006C007C004C00389828A8312141CE58124F5F5818061AE2A7F008E828F8315
:202CFD00A3122A68AD82AE83AFF0E52A242FF582E43400F583E0FC7B00E52A2401F582E422
:202D1D003400F583E0F97A00E924F3F9EA34FFFAE4C0E0740CC0E074FFC0E0C0E0E4C0E0AC
:202D3D00C0E0C005C006C007C004C00389828A8312141CE58124F5F581052A74D2252A40AA
:202D5D0003022C6E22E4C0E0744CC0E07473C0E0E4C0E0C0E004C0E0E4C0E0742FC0E0E4B7
:202D7D00C0E07460C0E07451C0E07480C0E07582041214C1E58124F4F581AE1B7F008E82FB
:202D9D008F83122A68AD82AE83AFF0E4C0E0740CC0E0744CC0E07473C0E0E4C0E0C0E0C0F2
:202DBD0005C006C00704C0E0E4C0E090006112141CE58124F5F58122E51E7003F51F2274D2
:202DDD0001B51E04851D1F22E51D75F00AA4251CF51F22E4C0E0740CC0E0744CC0E07473A4
:202DFD00C0E0E4C0E0C0E07424C0E0746EC0E07480C0E074E2C0E0E4C0E09000F912141C5F
:202E1D00E58124F5F5819003E81200A9752B00E51B75F02EA424D3FEE5F034FFFFAC2B7D43
:202E3D0000EC2EF582ED3FF583E4C0E0120304158190000A1200A9052B74D2252B50D09042
:202E5D0003E81200A9744CC0E07473C0E074EFC0E0E4C0E0743FC0E07401C0E074E2C0E0E3
:202E7D00E4C0E09000F9122571E58124F8F581851B82022F9E752C01E51B75F02EA4FEAF11
:202E9D00F0AC2C7D00EC2EFEED3FFFEE24D2F582EF34FFF583120349AF82BF0105122A9078
:202EBD0080069000461200A99002581200A9052C74D1252C50C2752C0122AFB374FE5FF574
:202EDD00B3AFB474FE5FF5B4AFCB74FE5FF5CBAFCC74FE5FF5CCAFCB74FB5FF5CBAFCC7436
:202EFD00FB5FF5CCAFE174FE5FF5E1AFE274FE5FF5E2AFCB747F5FF5CBAFCC747F5FF5CC10
:202F1D00AF9174FE5FF591AF9274FE5FF592AF9174FD5FF591AF9274FD5FF592AF9174F78B
:202F3D005FF591AF9274F75FF592AF9174BF5FF591AF9274BF5FF592AF91747F5FF591AF84
:202F5D0092747F5FF592AF9574FE5FF595AF9674FE5FF596AF9574FD5FF595AF9674FD5FF6
:202F7D00F596AF9574FB5FF595AF9674FB5FF596AF9574BF5FF595AF9674BF5FF596D2EFEC
:202F9D0022AF82752D00EF75F02EA424D3FEE5F034FFFF7406B52D02801A7412B52D02801B
:202FBD00137421B52D02800C7425B52D0280057426B52D15C007C006C02D758203122B2276
:202FDD001581D006D00702308FAC2D7D00EC2EF582ED3FF583C007C006120349E582D0061D
:202FFD00D007601CAC2D7D00EC2EF582ED3FF583C007C006120349AD82D006D007BDFF143F
:20301D00C007C006C02D758200122B221581D006D007805EAC2D7D00EC2EF582ED3FF58317
:20303D00C007C006120349AD82D006D007BD0114C007C006C02D758201122B221581D0069D
:20305D00D007802EAC2D7D00EC2EF582ED3FF583C007C006120349AD82D006D007BD0212AB
:20307D00C007C006C02D758202122B221581D006D007052D74D2252D4003022FB022E4C06A
:20309D00E014C0E0C0E0E4C0E0C0E07410C0E0E4C0E0740FC0E0E4C0E07418C0E07451C0BB
:2030BD00E07480C0E07582031214C1E58124F4F581E4C0E014C0E0C0E0E4C0E0C0E0741E1C
:2030DD00C0E0E4C0E0740FC0E0E4C0E074D0C0E07450C0E07480C0E07582031214C1E581E5
:2030FD0024F4F581E4C0E014C0E0C0E0E4C0E0C0E0742CC0E0E4C0E0740FC0E0E4C0E0744A
:20311D0088C0E07450C0E07480C0E07582031214C1E58124F4F581E4C0E014C0E0C0E0E4E1
:20313D00C0E0C0E0743AC0E0E4C0E0740FC0E0E4C0E07440C0E07450C0E07480C0E0758276
:20315D00031214C1E58124F4F581E4C0E014C0E0C0E0E4C0E0C0E07448C0E0E4C0E0740F15
:20317D00C0E0E4C0E074F8C0E0744FC0E07480C0E07582031214C1E58124F4F581E4C0E0B2
:20319D0014C0E0C0E0E4C0E0C0E07456C0E0E4C0E0740FC0E0E4C0E074B0C0E0744FC0E0DE
:2031BD007480C0E07582031214C1E58124F4F581E4C0E014C0E0C0E07430C0E07484C0E0D5
:2031DD007464C0E0E4C0E0740FC0E0E4C0E07468C0E0744FC0E07480C0E07582031214C1DB
:2031FD00E58124F4F581E4C0E014C0E0C0E0E4C0E0C0E07472C0E0E4C0E0740FC0E0E4C0F1
:20321D00E07420C0E0744FC0E07480C0E07582031214C1E58124F4F581E4C0E014C0E0C0B9
:20323D00E0E4C0E0C0E07480C0E0E4C0E0740FC0E0E4C0E074D8C0E0744EC0E07480C0E0CC
:20325D007582031214C1E58124F4F581E4C0E014C0E0C0E0E4C0E0C0E0748EC0E0E4C0E05A
:20327D00740FC0E0E4C0E07490C0E0744EC0E07480C0E07582031214C1E58124F4F581E437
:20329D00C0E014C0E0C0E0E4C0E0C0E0749CC0E0E4C0E0740FC0E0E4C0E07448C0E0744E00
:2032BD00C0E07480C0E07582031214C1E58124F4F581E4C0E014C0E0C0E0E4C0E0C0E07478
:2032DD00AAC0E0E4C0E0740FC0E0E4C0E07400C0E0744EC0E07480C0E07582031214C1E58C
:2032FD008124F4F581E4C0E014C0E0C0E0E4C0E0C0E074B8C0E0E4C0E0740FC0E0E4C0E0AF
:20331D0074B8C0E0744DC0E07480C0E07582031214C1E58124F4F581E4C0E014C0E0C0E022
:20333D00E4C0E0C0E074C6C0E0E4C0E0740FC0E0E4C0E07470C0E0744DC0E07480C0E07559
:20335D0082031214C1E58124F4F581E4C0E014C0E0C0E0E4C0E0C0E074D4C0E0E4C0E07414
:20337D000FC0E0E4C0E07428C0E0744DC0E07480C0E07582031214C1E58124F4F581E4C053
:20339D00E014C0E0C0E0E4C0E0C0E074E2C0E0E4C0E0740FC0E0E4C0E074E0C0E0744CC023
:2033BD00E07480C0E07582031214C1E58124F4F581E4C0E014C0E0C0E0E4C0E0C0E0741027
:2033DD00C0E0E4C0E0745AC0E0E4C0E07498C0E0744CC0E07480C0E07582031214C1E581D3
:2033FD0024F4F581E4C0E014C0E0C0E0E4C0E0C0E0741EC0E0E4C0E0745AC0E0E4C0E0740A
:20341D0050C0E0744CC0E07480C0E07582031214C1E58124F4F581E4C0E014C0E0C0E0748A
:20343D0030C0E07484C0E0742CC0E0E4C0E07460C0E0E4C0E07420C0E0744CC0E07480C003
:20345D00E07582021214C1E58124F4F581E4C0E014C0E0C0E0E4C0E0C0E0743AC0E0E4C0AD
:20347D00E0745AC0E0E4C0E074D8C0E0744BC0E07480C0E07582031214C1E58124F4F581A9
:20349D00E4C0E014C0E0C0E0E4C0E0C0E07448C0E0E4C0E07460C0E0E4C0E074A8C0E0740B
:2034BD004BC0E07480C0E07582021214C1E58124F4F581E4C0E014C0E0C0E0E4C0E0C0E0A0
:2034DD007456C0E0E4C0E0745AC0E0E4C0E07460C0E0744BC0E07480C0E07582031214C1A7
:2034FD00E58124F4F581E4C0E014C0E0C0E0E4C0E0C0E07464C0E0E4C0E0745AC0E0E4C0B1
:20351D00E07418C0E0744BC0E07480C0E07582031214C1E58124F4F581E4C0E014C0E0C0C2
:20353D00E0E4C0E0C0E07472C0E0E4C0E07460C0E0E4C0E074E8C0E0744AC0E07480C0E07A
:20355D007582021214C1E58124F4F581E4C0E014C0E0C0E0E4C0E0C0E07480C0E0E4C0E066
:20357D00745AC0E0E4C0E074A0C0E0744AC0E07480C0E07582031214C1E58124F4F581E4DD
:20359D00C0E014C0E0C0E0E4C0E0C0E0748EC0E0E4C0E0745AC0E0E4C0E07458C0E0744AB4
:2035BD00C0E07480C0E07582031214C1E58124F4F581E4C0E014C0E0C0E0E4C0E0C0E07475
:2035DD009CC0E0E4C0E0745AC0E0E4C0E07410C0E0744AC0E07480C0E07582031214C1E540
:2035FD008124F4F581E4C0E014C0E0C0E0E4C0E0C0E074AAC0E0E4C0E0745AC0E0E4C0E06F
:20361D0074C8C0E07449C0E07480C0E07582031214C1E58124F4F581E4C0E014C0E0C0E013
:20363D00E4C0E0C0E074B8C0E0E4C0E0745AC0E0E4C0E07480C0E07449C0E07480C0E0750D
:20365D0082031214C1E58124F4F581E4C0E014C0E0C0E0E4C0E0C0E074C6C0E0E4C0E0741F
:20367D005AC0E0E4C0E07438C0E07449C0E07480C0E07582031214C1E58124F4F581E4C0F9
:20369D00E014C0E0C0E0E4C0E0C0E074D4C0E0E4C0E0745AC0E0E4C0E074F0C0E07448C0D7
:2036BD00E07480C0E07582031214C1E58124F4F581E4C0E014C0E0C0E0E4C0E0C0E074E252
:2036DD00C0E0E4C0E0745AC0E0E4C0E074A8C0E07448C0E07480C0E07582031214C1E581C4
:2036FD0024F4F581E4C0E014C0E0C0E0E4C0E0C0E07410C0E0E4C0E074A5C0E0E4C0E074CA
:20371D0060C0E07448C0E07480C0E07582031214C1E58124F4F581E4C0E014C0E0C0E0747B
:20373D0030C0E07484C0E0741EC0E0E4C0E074A5C0E0E4C0E07418C0E07448C0E07480C0D5
:20375D00E07582031214C1E58124F4F581E4C0E014C0E0C0E0E4C0E0C0E0742CC0E0E4C0B7
:20377D00E074A5C0E0E4C0E074D0C0E07447C0E07480C0E07582031214C1E58124F4F58167
:20379D00E4C0E014C0E0C0E0E4C0E0C0E0743AC0E0E4C0E074A5C0E0E4C0E07488C0E074F1
:2037BD0047C0E07480C0E07582031214C1E58124F4F581E4C0E014C0E0C0E0E4C0E0C0E0A0
:2037DD007448C0E0E4C0E074A5C0E0E4C0E07440C0E07447C0E07480C0E07582031214C18B
:2037FD00E58124F4F581E4C0E014C0E0C0E07430C0E07484C0E07456C0E0E4C0E074A5C03D
:20381D00E0E4C0E074F8C0E07446C0E07480C0E07582031214C1E58124F4F581E4C0E014C0
:20383D00C0E0C0E07430C0E07484C0E07464C0E0E4C0E074A5C0E0E4C0E074B0C0E0744698
:20385D00C0E07480C0E07582031214C1E58124F4F581E4C0E014C0E0C0E0E4C0E0C0E074D2
:20387D0072C0E0E4C0E074A5C0E0E4C0E07468C0E07446C0E07480C0E07582031214C1E528
:20389D008124F4F581E4C0E014C0E0C0E0E4C0E0C0E07480C0E0E4C0E074A5C0E0E4C0E0AB
:2038BD007420C0E07446C0E07480C0E07582031214C1E58124F4F581E4C0E014C0E0C0E01C
:2038DD00E4C0E0C0E0748EC0E0E4C0E074A5C0E0E4C0E074D8C0E07445C0E07480C0E075F6
:2038FD0082031214C1E58124F4F581E4C0E014C0E0C0E0E4C0E0C0E0749CC0E0E4C0E074A7
:20391D00A5C0E0E4C0E07490C0E07445C0E07480C0E07582031214C1E58124F4F581E4C0B7
:20393D00E014C0E0C0E0E4C0E0C0E074AAC0E0E4C0E074A5C0E0E4C0E07448C0E07445C0BE
:20395D00E07480C0E07582031214C1E58124F4F581E4C0E014C0E0C0E0E4C0E0C0E074B8D9
:20397D00C0E0E4C0E074A5C0E0E4C0E07400C0E07445C0E07480C0E07582031214C1E58181
:20399D0024F4F581E4C0E014C0E0C0E0E4C0E0C0E074C6C0E0E4C0E074A5C0E0E4C0E07471
:2039BD00B8C0E07444C0E07480C0E07582031214C1E58124F4F58122A2F822120301900746
:2039DD00D012034985821B7440C0E07401C0E09000F012085A1581158175820312059375D8
:2039FD008203120B4790FFFF120BDC9007D1120349AF82BF0103023A8CE4C0E07420C0E000
:203A1D0074FFC0E0C0E0E4C0E0C0E0742CC0E0746EC0E07480C0E07464C0E0E4C0E09000D0
:203A3D001E12141CE58124F5F5819027101200A990FFFF120BDCE4C0E014C0E0C0E0E4C08F
:203A5D00E0C0E07464C0E0E4C0E0741EC0E0E4C0E074B8C0E07442C0E07480C0E075820466
:203A7D00121B6FE58124F4F5819003E81200A990FFFF120BDC744CC0E07473C0E0740EC0B3
:203A9D00E0E4C0E0743FC0E07401C0E0E4C0E0C0E0900000122571E58124F8F581744CC069
:203ABD00E07473C0E074EFC0E0E4C0E0743FC0E07401C0E0E4C0E0C0E09000F7122571E55B
:203ADD008124F8F581122ED7122A9012309B122C6B851B82122F9E022D62122DD5122AB0BB
:203AFD00D297C2901239D520A0299000141200A930A003023BD77401B51E08751C01751E2A
:203B1D0002800AE51E7006751D01751E0130A0FD023BD720A1299000141200A930A103025C
:203B3D003BD77401B51E08751C02751E02800AE51E7006751D02751E0130A1FD023BD720B1
:203B5D00A2289000141200A930A203023BD77401B51E08751C03751E02800AE51E70067545
:203B7D001D03751E0130A2FD805020A64D9000141200A920A6447401B51E0B751E00751CE2
:203B9D0000751D0080317402B51E2C751E01751C00744CC0E07473C0E0740EC0E0E4C0E09E
:203BBD007428C0E0E4C0E0C0E0C0E0900021122571E58124F8F58130A6FD9000051200A974
:203BDD00D290C2911239D520A0299000141200A930A003023CBA7401B51E08751C04751E68
:203BFD0002800AE51E7006751D04751E0130A0FD023CBA20A1299000141200A930A1030295
:203C1D003CBA7401B51E08751C05751E02800AE51E7006751D05751E0130A1FD023CBA2002
:203C3D00A2289000141200A930A203023CBA7401B51E08751C06751E02800AE51E7006757D
:203C5D001D06751E0130A2FD805320A6509000141200A920A647051BE51B24F55029751B2A
:203C7D0001744CC0E07473C0E0740EC0E0E4C0E0746EC0E0E4C0E0C0E0C0E0900067122525
:203C9D0071E58124F8F581C01B9007D01203041581122D62851B82122F9E30A6FD900005A3
:203CBD001200A9D291C2931239D520A0299000141200A930A003023DA27401B51E08751C77
:203CDD0007751E02800AE51E7006751D07751E0130A0FD023DA220A1299000141200A930D4
:203CFD00A103023DA27401B51E08751C08751E02800AE51E7006751D08751E0130A1FD02A3
:203D1D003DA220A2289000141200A930A203023DA27401B51E08751C09751E02800AE51E9C
:203D3D007006751D09751E0130A2FD805820A6559000141200A920A64C151B74FF251B406B
:203D5D0003751B0A7409B51B26744CC0E07473C0E0740EC0E0E4C0E0746EC0E0E4C0E0C0E3
:203D7D00E0C0E0900067122571E58124F8F581C01B9007D01203041581122D62851B821249
:203D9D002F9E30A6FD9000051200A9D293C2961239D530A003023E2E9000141200A930A0C9
:203DBD0003023EE9E51B75F02EA4FEAFF0AC1F7D00EC2EFEED3FFFEE24D2F582EF34FFF5E9
:203DDD00837401C0E01203041581751F00751C00E4F51DF51EC0E0758201122B221581853F
:203DFD001B82122F9E744CC0E07473C0E0740EC0E0E4C0E07428C0E0E4C0E0C0E0C0E0900D
:203E1D00001A122571E58124F8F58130A0FD023EE920A1289000141200A930A103023EE990
:203E3D007401B51E08751C00751E028009E51E7005F51D751E0130A1FD023EE930A203027A
:203E5D003ED79000141200A930A203023EE9E51B75F02EA4FEAFF0AC1F7D00EC2EFEED3F73
:203E7D00FFEE24D2F582EF34FFF58374FFC0E01203041581751F00751C00E4F51DF51EC081
:203E9D00E0758200122B221581851B82122F9E744CC0E07473C0E0740EC0E0E4C0E074280F
:203EBD00C0E0E4C0E0C0E0C0E090001A122571E58124F8F58130A2FD801220A60F9003E886
:203EDD001200A920A606122DF030A6FD9000051200A9D296C2971239D530A003023F7490F3
:203EFD0000141200A930A003023FB1E51B75F02EA4FEAFF0AC1F7D00EC2EFEED3FFFEE24A0
:203F1D00D2F582EF34FFF5837402C0E01203041581751F00751C00E4F51DF51EC0E0758217
:203F3D0002122B221581851B82122F9E744CC0E07473C0E0740EC0E0E4C0E07428C0E0E4BF
:203F5D00C0E0C0E0C0E090001A122571E58124F8F58130A0FD803D20A12B9000141200A945
:203F7D0020A131C2EF9003E81200A9D2EF9003E81200A9C2EF122E929003E81200A9D2EFDA
:203F9D0030A1FD800F20A20C9000141200A920A20330A2FD9000050200A91239D8123AF740
:023FBD0080FB87
:2042B80000000000000000100200003002200060023001C0021C0380020E0E000207BC00AB
:2042D8000201F0000207F002027FF80203FC3F060FE00FC4070007CC0201801800070030AB
:2042F800003C006001F001C03FE007807FC03F0038DFFC0000DFE00000DFE00000C0FE00E5
:2043180000C00F8000C001E000CC00F000F8003800F0001C01E0000C00C0000C00000000E4
:2043380000000000000800200008007000080070600800E0300801C03C1FFF801E3FFF8056
:204358000E180080000800C0000000600000003007FFFC3007FFFC1804001C180C00181887
:204378000C00301C1800201C3800601C3800401C37FFFFDC07FFFFDC07FFFF9C0600001C7C
:204398000600081C06000C1C06000E1C07FFFE1C0FFFFC1C07FFF018000000100000001009
:2043B80000000000000040000000C0000001800000070000001C00000078000001FFFFFECC
:2043D8000FFFFFFE7F3000007C0000013000000203000002033FF006033FE004033FE80CC3
:2043F80003304718033043B8033040F003304FE07FFFFFF07FFFFC38233040180330400CD7
:204418000330400C0330400E033FE00E037FE006073FE006070000060300000400000004A8
:2044380000000000000000020000000400000018000000F03FFFFFE03FFFFF001FFFF800E6
:20445800101030001010300010103000101030001010300010103000101030001FFFFFFCFB
:204478001FFFFFFC1FFFFFFC10103000101030001010300010103018101030181010300CD6
:204498001010300E1010300E3FFFFFFE3FFFFFFC10000000000000000000000000000000C4
:2044B800110CFFEC110C080C7F8C088C48CC48AC50AC908C208C470C200C200C3F8C208C1E
:2044D800410C410C820C040C0A0C110C208CC06C010CEFECA10CA7CCA10CEFECA44CA7CC8E
:2044F800A44CE7CCA44C04CC202C102C012CFD2C092C092C492C292C112C282C442C84ECBE
:20451800210C210C23ECAC0CA80CABCCA84CA88CA90CBA2CCA2C01EC040CFFEC802C7FCC9F
:20453800400C5F8C400C7FCC522C514C548C986C200C2FCC420C420CC20C4FCC424C424CCE
:20455800444C444C444C5FEC200C27EC224CF24C524C57EC524C924C524C244C544C884C7E
:20457800014CF90C13EC528C968CFBEC328C528C53EC928C128C33EC040C7FCC080C3F8CFB
:20459800100CFFEC208C5F4C842C7FCC150C248C7FCC404C7FCC404C7FCC014C7FEC412CBB
:2045B8007D4C44AC4D6C822CF90C890CF90C03ECF92C892CA92CA92CA92C222C522C8CCCB8
:2045D8003FEC202C222C2FAC222C3FEC202C2FAC28AC2FAC402C80EC090C088CFFEC128CCA
:2045F800232CCDEC110C7FCC110CFFEC208C404C000C3F8C010C020C040C040CFFEC040CE6
:20461800040C040C040C1C0C020CF24C128C130CF20C87EC828CF28C124C124C132C620CBB
:20463800010CF10C2FEC210C27CCF10C2FEC212C212C316CC10C010C040CFFEC802C7FCC02
:20465800400C5F8C400C7FCC522C514C548C986C040C7FCC040CFFEC000C7FCC404C7FCCF1
:20467800122C314CD48C186C000C3F8C010C020C040C040CFFEC040C040C040C040C1C0C1E
:20469800200C27CCF10C410CA10CF10C2FEC310CE10C210C210C210C228C228C2AACF6CC2F
:2046B800528C528C56CC9AAC528C22AC54AC886C7FCC404C7FCC404C7FCC040C440C7FCC7A
:2046D800840C3F8C040CFFEC000C7FEC400C5FCC400C7FEC490C492C494C488C4C4C882C48
:2046F800000C7FCC040C040C040C040C7FCC040C040C040C040CFFEC040C020C3FEC202C00
:20471800202C3FEC200C3FEC302C502C5FEC902C410C410C73EC842CEA4C418C420CF7ECF7
:204738004A2C422C63EC422C200C27CC208CF90C220C67EC72ACAAAC252C292C222C24CC17
:20475800210C450CF7CC990C910C9FECF00C97CC944C944CF7CC944C000C7FEC400C5FCC83
:20477800400C7FEC490C492C494C488C4C4C882C214C458C7D2C00EC7C0C452C7D4C458C85
:204798007D2C44EC524C892C000C03CC7C0C040C040C040CFFEC040C040C040C040C040C07
:2047B800208C210C27ECF42C242C742C6FECA42C242C242C27EC242C884C5E4C124C1EECD1
:2047D800D24C5E4C534C7ECC4A4C524C624C46CC9FCC488C050C020C0D8CB26C420C1FCCCE
:2047F800020C3FEC420C820C220C23CC444C538CDC6C508C510C564C518C562C40CC4F0C17
:20481800200C27CC208CF90C220C67EC72ACAAAC252C292C222C24CC000C3F8C010C020CE5
:20483800040C040CFFEC040C040C040C040C1C0C17CC924C918C924C142C000C7FCC444C0A
:20485800444C0B0C30CCC02C020C820C5FEC122C122C820C450C050C090C492C912C20EC0B
:2048780021CCF94C894C526CFC0C21CCD54C294CDD4C288CC94C322C9F8C408C010C222C2E
:20489800AAAC672C222C272C2AAC622CA62C3FEC7F8C008C208C208C208C3FEC002C002CF7
:2048B800FFAC002C002C01CC410C210CF7EC110C23CC210C77ECA92C212C216C210C210C0E
:2048D800000CF7EC942C942CA42CA7EC942C942C942CE42C87EC842C040C07EC040C040C58
:2048F8007FCC404C404C7FCC404C400C400C800C000C080C040C020C120C104C502C502C92
:20491800502C908C108C0F8C080C040CFFEC802C802C3F8C040C040CFFEC040C040C1C0C2B
:20493800202C102C012CFD2C092C092C492C292C112C282C442C84EC044CF44C2FEC244CC1
:2049580027CCF44C27CC244C2FEC300CC44C082C200C27CCF10C410CA10CF10C2FEC310CA3
:20497800E10C210C210C210C202C102C012CFD2C092C092C492C292C112C282C442C84EC28
:20499800010C890C4FCC110C010C9FEC400C0FCC284C484C8FCC084C000C7FEC400C5FCCC1
:2049B800400C7FEC490C492C494C488C4C4C882C038C7C0C400C440C440C7FCC040C248C9B
:2049D800244C442C842C1C0C000C3F8C010C020C040C040CFFEC040C040C040C040C1C0CA2
:2049F80027EC242C2FECB42CA7ECA10CA08C27EC200C542C524C8FEC110C7FCC110CFFEC8D
:204A1800040C7FCC444C7FCC444C7FCC208C404C000C7FCC208C110C0E0C318CC46C040CFE
:204A38003F8C040C040CFFEC208C208CFBEC208C208CFBEC000CFBEC8A2C8A2CFBEC8A2C0E
:204A5800100CFDEC012C7D2C454C7D4C012C792C092CFDCC110C310C080C080C1FCC204C60
:204A7800508C0B0C0C0C3FECD02C102C1FEC102C010C890C4FCC110C010C9FEC400C0FCCD0
:204A9800284C484C8FCC084C110CFFEC110C3FCC204C3FCC204C7FEC442CAA2C3FAC006C2C
:204AB8007FCC404C7FCC404C7FCC200C3FEC492C892C122C242C49CC080C040CFFEC000CA6
:204AD8007FCC000C7FCC000C7FCC404C7FCC404C228C3FEC420C5FCCD24C5FCC524C524C8B
:204AF800408C5FEC488C458C7FCC008C190C060C010CFFEC042C044C048C040C040C1C0C84
:204B18003FEC202C222C2FAC222C3FEC202C2FAC28AC2FAC402C80EC044CF44C2FEC244C9B
:204B380027CCF44C27CC244C2FEC300CC44C082C00ECEF0C422C494C440CE7CC490C410C9D
:204B58004FEC610CC92C0FEC3FEC202C222C2FAC222C3FEC202C2FAC28AC2FAC402C80ECDE
:204B7800080CE80C48EC5EAC4AACEAAC4AAC4AAC4AAC6AACD2EC26AC200C2FCC424C424C80
:204B9800DFEC424C424C4FCC424C420C440C480C440C29EC012C7D2C114C114CFF2C112C1E
:204BB800292C25CC450C810C200C27CC204CF88C490C490C4FEC910C510C210C510C8B0CAA
:204BD800020CF24C128C130CF20C87EC828CF28C124C124C132C620C0D0C710C41EC412C1E
:204BF8007E4C480C488C488C488C494C494C8A2C214C392C490C6FEC910C528C228C444CE8
:204C1800882C000C524C892C020CF24C128C130CF20C87EC828CF28C124C124C132C620CFA
:204C3800080CEFECB42CA7ACCA2CC22CBFACA22CAAACCFAC802C80CC040C0A0C110C208C65
:204C5800DF6C040C040C7FCC040C248C444C8C2C210C2FEC282CF40C56EC5AAC5AAC96EC12
:204C7800528C24AC54AC886C000C7FEC400C5FCC400C7FEC490C492C494C488C4C4C882C56
:204C9800200C27CC208CF90C220C67EC72ACAAAC252C292C222C24CC7FCC444C444C7FCC9D
:204CB800444C444C7FCC040C524C522C90AC0F8C040CFFEC040C7FCC208C3F8C110CFFEC99
:204CD800200CFDEC252CCDEC210C428C844C182C27CC610CAFEC210C254C252C292C230C20
:204CF800000C3F8C010C020C040C040CFFEC040C040C040C040C1C0C884C484C3FEC084C50
:204D18008FCC484C0FCC084C3FEC400C884C102C210C428C844C182C27CC610CAFEC210C9F
:204D3800254C252C292C230C108C108C210C3DEC524C944C104C104C104C104C104C11CC60
:204D5800040C7FEC108C090C7FEC410C460C58CC430C5C6C438C9C0C210C428C844C182C44
:204D780027CC610CAFEC210C254C252C292C230C410C2FEC010CF7CC010C9FEC544C57CC1A
:204D9800044C37CCC44C04CC040C7FCC110CFFEC444C7FCC444C7FCC040C7FCC040CFFEC59
:204DB800000C7FCC040C040C040C040C7FCC040C040C040C040CFFEC220CFB8C248C790CE4
:204DD80027CCF94C57EC714C57CC714C510C530C200C27EC224CF24C524C57EC524C924C9F
:204DF800524C244C544C884C000C9FCC420C020C020C820C5FCC020C220C420C820C3FEC3C
:204E1800000C080C040C020C120C104C502C502C502C908C108C0F8C210C210C220CB44C73
:204E3800AFECA02CA7CC244C244C244C27CC244C010CF10C110C110C254C254C352CE52C35
:204E5800292C210C210C630C9FEC420C0FCC044CC44C5FEC400C4FCC484C684C4FCC084C9F
:204E7800110CFFEC150C040CFFEC080C100C3FCC504C904C1FCC104C080C040CFFEC802C41
:204E9800040C040CFFEC0E0C150C248CC46C040C080C040CFFEC110C514C912C230C040CFF
:204EB800FFEC0A0C318CC06C3FCC204C3FCC204C7FEC400C5FCC400C7FEC524C518C986CEA
:204ED800110C510C520C7BEC944C124C1A4CF28C110C128C144C182C044CEFEC444C47CC2C
:204EF800410CEFEC492C4FEC410C6FECC10C0FEC208CFFEC248CFFEC802C7FCC404C7FCC52
:204F1800404C7FCC000CFFEC3F8C208C208C208C3F8C000C7FCC404C404C404C7FCC404C3F
:204F3800110CFFEC150C040CFFEC080C100C3FCC504C904C1FCC104C040C040C7FCC444C40
:204F5800444C7FCC444C444CFFEC404C404C41CC090C088C080CFFEC0A0C120C124C128C56
:204F7800230C222C462C89EC038C7C0C400C440C440C7FCC040C248C244C442C842C1C0CEF
:204F98003FCC204C3FCC204C7FEC400C5FCC400C7FEC524C518C986C202C102C012CFD2C15
:204FB800092C092C492C292C112C282C442C84EC220C210C27CCF00C244C728C6FECA10C74
:204FD80027CC210C210C210C208CFFEC248CFFEC802C7FCC404C7FCC404C7FCC000CFFEC71
:204FF8004F8C228C8ACC52AC048C498C840CFFEC150C248CC46C040C088CABEC514C2A2CAD
:205018000FEC882C5BAC2AAC0AAC4BAC8A2C306C3FCC204C3FCC204C7FEC400C5FCC400CD1
:205038007FEC524C518C986C110CFFEC110C240CAFCC748C230C2C8C7FECA88C248C218CBB
:20505800110C110C27CC210C610CAFEC200C210C27CC210C210C2FEC248CFA8C20ECF92CAE
:205078008A8C748C514C722C008C520C26ACF9AC210CF90C27ECF90C8BCCF90C8FECF92C20
:20509800212CF96C210C210C038C7C0C400C440C440C7FCC040C248C244C442C842C1C0C26
:2050B800200C2FCC424C424CDFEC424C424C4FCC424C420C440C480C000CFBEC808CB90C4F
:2050D800ABECAA2CAAACBAACA2ACA88CB14C222C440C27CC084C148C830C5CEC000C0FCCCD
:2050F800284C484C8FCC084C200C27CC204CF28C510C5FEC512C910C510C210C510C8B0C98
:20511800080C040C000CFFEC040C040C050C048C044C040C040C040C11CCFD4C13EC7D4C2D
:20513800548C7F6C950C3F8C60CCBFAC208C3F8C00ECEF0C422C494C440CE7CC490C410C83
:205158004FEC610CC92C0FEC040C444C248C040C7FCC004C004C3FCC004C004C7FCC004C22
:20517800208C110CFFEC000C7C4C454C7D4C454C7D4C454C444C4CCCFFEC040C080C7FCC48
:20519800404C404C444C444C444C0B0C30CCC02C0FCCF04C244C244C444C77ECD02C502CCE
:2051B8005FAC702C502C00CC210C228CF44C4BACA00CFE2C2AAC3EACEAAC2EAC2A2C2A6CE4
:2051D800300C080C040C040C0A0C0A0C0A0C110C110C208C404C802C0000000000000000E7
:2051F8000000000000000404040404040004000000140A0A0000000000000000000014142B
:205218003F140A3F0A0A000000041E1505060C14150F0400000012150D0A142C2A12000082
:205238000000040A0A1E15150936000000020201000000000000000000201008080808085A
:205258000810200000020408080808080804020000000004150E0E1504000000000004046C
:20527800041F04040400000000000000000000000002020100000000001F000000000000C3
:2052980000000000000000000002000000100808080404020202010000000E11111111115A
:2052B800110E00000000040604040404040E000000000E1111080402011F000000000E110E
:2052D800100C1010110E00000000080C0A0A091E0818000000001F01010F1010110E00007D
:2052F80000000E09010F1111110E000000001F09080404040404000000000E11110E11118A
:20531800110E000000000E1111111E10120E000000000000040000000004000000000000BF
:205338000004000000040400002010080402040810200000000000001F00001F0000000091
:2053580000020408102010080402000000000E11110804040004000000000E111915151D16
:20537800011E0000000004040C0A0A1E1233000000000F12120E1212120F000000001E11B6
:2053980001010101110E000000000F1212121212120F000000001F120A0E0A02121F0000C2
:2053B80000001F120A0E0A020207000000001C1201013911120C000000003312121E121246
:2053D8001233000000001F0404040404041F000000003E0808080808080907000000371253
:2053F8000A060A0A123700000000070202020202223F000000001B1B1B1B151515150000F6
:2054180000003B1216161A1A1217000000000E1111111111110E000000000F12120E0202D7
:205438000207000000000E1111111117190E180000000F12120E0A121237000000001E11CE
:2054580001060810110F000000001F1504040404040E00000000331212121212120C0000F4
:2054780000003312120A0A0C0404000000001515150E0A0A0A0A000000001B0A0A04040ADF
:205498000A1B000000001B0A0A040404040E000000001F0908040402121F0000001C0404F3
:2054B8000404040404041C00000202020404080808100000000E08080808080808080E000E
:2054D80000040A00000000000000000000000000000000000000003F000400000000000063
:2054F8000000000000000000000C121C123C000000000302020E1212120E000000000000B3
:20551800001C1202021C000000001810101C1212123C000000000000000C121E021C000005
:2055380000003804041E0404041E000000000000003C120C021E221C00000302020E1212DA
:20555800123700000000040000060404040E000000000800000C080808080807000003027E
:20557800023A0A0E123700000000070404040404041F000000000000000F151515150000D5
:2055980000000000000F12121237000000000000000C1212120C000000000000000F1212F6
:2055B800120E020700000000001C1212121C103800000000001B06020207000000000000C8
:2055D800001E020C101E000000000004040E04040418000000000000001B1212123C000092
:2055F800000000000037120A0C040000000000000015150E0A0A000000000000001B0A04BB
:205618000A1B0000000000000037120A0C04040300000000001E0804041E0000001808086F
:2056380008040808080818000808080808080808080808080006040404080404040406007E
:205658000225180000000000000000000000000000000000000000000000000000000000F3
:20567800000000000000000000000000000000000000000000000000000000000000000012
:20569800000000000000000000000000000000000000000000000000C003C003C003C003E6
:2056B800C003C0038003800180018001800180018001800180010000000000008001C0037D
:2056D800C0038001000000000000000000000000C018E01CE01C700E300618038C018400BE
:2056F800000000000000000000000000000000000000000000000000000000000000000092
:205718000000000000000000000000000000000000000000000000002010201020102010B1
:205738002010FE7FFE7FFE7F100810081008100810081008FE7FFE7FFE7F180C0804080467
:20575800080408040000000000000000000000000000000080008000C003B00C9018981842
:20577800981C981CB800B000F000E000C0038007800F800C801C80189C189C188C188C0C34
:205798009806E00380008000800000000000000000000000000000001C0836082204630401
:2057B800630263026302630163012201B61C9C36402240634063206320631063106310224D
:2057D8000836081C0000000000000000000000000000000000000000F00098008C018C01AD
:2057F8008C018C018C00CC005C0038001C3E3C08320873086304E304C3048303834306676A
:205818008C3E781C0000000000000000000000001C003C003C003000300010000C000600FC
:20583800000000000000000000000000000000000000000000000000000000000000000050
:20585800000000000000000000000000000000000040002000100018000C00040006000290
:2058780000030003800180018001800180018001800180018001000300030002000600046F
:20589800000C00180010002000400000000000000200040008001800300020006000400046
:2058B800C000C000800180018001800180018001800180018001C000C000C0006000200007
:2058D8003000180008000400020000000000000000000000000000000000000000038003D4
:2058F80080030C631C713839600D80038003600D38391C718C61800380038003000000004C
:2059180000000000000000000000000000000000000000000000000000000000000000016E
:20593800000100010001000100010001FC7F000100010001000100010001000100000000C7
:2059580000000000000000000000000000000000000000000000000000000000000000002F
:20597800000000000000000000000000000000000000000000000000000000001C003C00B7
:205998003C003000300010000C000600000000000000000000000000000000000000000031
:2059B800000000000000000000000000FE7F00000000000000000000000000000000000052
:2059D8000000000000000000000000000000000000000000000000000000000000000000AF
:2059F8000000000000000000000000000000000000000000000000000000000018003C003B
:205A18003C00180000000000000000000000000000000040006000200030001000180008FA
:205A3800000C0004000600020003000180018000C000400060002000300010001800080051
:205A58000C0004000600020000000000000000000000000000000000C0036004300C181883
:205A7800181818100C300C300C300C300C300C300C300C300C300C30181018181818300C9A
:205A98006004C003000000000000000000000000000000000000000000018001F8018001CB
:205AB8008001800180018001800180018001800180018001800180018001800180018001BE
:205AD800C003F81F0000000000000000000000000000000000000000E007101C081804306D
:205AF80004300C300C30003000180018000C000600038001C0004000202010200820043020
:205B1800FC1FFC1F0000000000000000000000000000000000000000E00318060C0C0C18FA
:205B38000C180C1800180018000C0006C003000E00180010003000300C300C300C100C18B2
:205B5800180CE003000000000000000000000000000000000000000000060006000700070C
:205B7800800680064006200620061006100608060C0604060206FE3F0006000600060006BC
:205B98000006C03F0000000000000000000000000000000000000000F03FF03F080008007A
:205BB8000800080008000800C807280C1818081000300030003000300C300C3004180418F2
:205BD800180CE0030000000000000000000000000000000000000000800760183018101837
:205BF8001800080008000C00CC076C0C1C181C100C300C300C300C300C30183018103018CA
:205C1800700CC0070000000000000000000000000000000000000000F83FF83F08100C088F
:205C3800040804040004000200020002000100018000800080008000C000C000C000C0002C
:205C5800C000C0000000000000000000000000000000000000000000E007300C18180C301D
:205C78000C300C301C301C107818F004E003180F0C1E0C1C063806300630063006300C1802
:205C9800180CE0030000000000000000000000000000000000000000E00318040C080C18AE
:205CB8000610063006300630063006300E380C341836F03100300018001800080C0C0C0621
:205CD8000C03F00100000000000000000000000000000000000000000000000000000000AC
:205CF8000000000000008001C003C003800100000000000000000000000000008001C003C0
:205D1800C00380010000000000000000000000000000000000000000000000000000000027
:205D38000000000000000000C001C001C00100000000000000000000000000000000C00147
:205D5800C001C0018001C000C000000000000000000000000000000000200010000800046C
:205D7800000200018000400020001000080008001000200040008000000100020004000809
:205D98000010002000000000000000000000000000000000000000000000000000000000BB
:205DB800000000000000FE7F00000000000000000000FE7F000000000000000000000000D1
:205DD80000000000000000000000000000000000000000000000000004000800100020006F
:205DF80040008000000100020004000800100010000800040002000180004000200010009D
:205E1800080004000000000000000000000000000000000000000000C0073018183008609F
:205E38000C601C601C601C6000300018000E00030001000100010001000000008001C003C9
:205E5800C00380010000000000000000000000000000000000000000C0076008301018203F
:205E78000C2B8C4D844CC64CC6446644664466446646662666266417CC0C0C40082018303D
:205E98003018C0070000000000000000000000000000000000000000C001C001C001C001D7
:205EB800200320032003200330021006100610061804F80F080C080C080C04180418041817
:205ED80006381F7C0000000000000000000000000000000000000000FE07181C1818183020
:205EF80018301830183018301818180CF807181818301820186018601860186018601830C7
:205F18001818FE0F0000000000000000000000000000000000000000C00760381030186015
:205F38000C400C400C000600060006000600060006000600060006000C400C400820181087
:205F58003008C0070000000000000000000000000000000000000000FE03180E18181810AB
:205F7800183018301860186018601860186018601860186018601820183018301818181819
:205F98001806FE030000000000000000000000000000000000000000FE3F183018201840B5
:205FB80018401800180018081808180CF80F180C1808180818001800180018401840182042
:205FD8001830FE3F0000000000000000000000000000000000000000FE3F18381820184007
:205FF80018401800180018081808180CF80F180C180818081808180018001800180018009A
:2060180018007E000000000000000000000000000000000000000000C003300C100818188B
:206038000C100C10040006000600060006000600067E0618061804180C180C18081818187A
:206058003004E00300000000000000000000000000000000000000003FFC0C300C300C3022
:206078000C300C300C300C300C300C30FC3F0C300C300C300C300C300C300C300C300C3049
:206098000C303FFC0000000000000000000000000000000000000000F81F800180018001D7
:2060B8008001800180018001800180018001800180018001800180018001800180018001B8
:2060D8008001F81F0000000000000000000000000000000000000000E07F0006000600069F
:2060F800000600060006000600060006000600060006000600060006000600060006000628
:20611800000600060E060E038E01FC000000000000000000000000007E3E180C1804180691
:2061380018021801180198009800D800B801B8011803180318061806180C180C180C181873
:2061580018187E7C00000000000000000000000000000000000000007E0018001800180037
:206178001800180018001800180018001800180018001800180018001800184018401820E7
:206198001830FE3F00000000000000000000000000000000000000000FF01C381C381C3867
:2061B8001C381C343434343434343432343264326432643264314431C431C431C430C43081
:2061D80084308FFC00000000000000000000000000000000000000000FF81C201C20342095
:2061F800342064206420C420C420842184210423042304260426042C042C0438043804306B
:2062180004301F200000000000000000000000000000000000000000C003300C18180810AC
:206238000C300C3006200660066006600660066006600660066004600C300C300810181854
:20625800300CC0030000000000000000000000000000000000000000FE0F1818183018602A
:206278001860186018601860186018301818F8071800180018001800180018001800180077
:2062980018007E000000000000000000000000000000000000000000C003300C1818081009
:2062B8000C300C300660066006600660066006600660066006600660E4211C331C36181E76
:2062D800300EC007004C003C00380000000000000000000000000000FE07181C1818183030
:2062F80018301830183018301818180CF80718031803180618061806180C180C180C1818E7
:2063180018187E780000000000000000000000000000000000000000F013181E0C180618C4
:206338000610061006000E003C00F800E003800F001E0018003802300230063004300C18FF
:206358001C0CE4070000000000000000000000000000000000000000FC3F8C218461824182
:206378008241800180018001800180018001800180018001800180018001800180018001B3
:206398008001E00700000000000000000000000000000000000000003F7C0C100C100C106E
:2063B8000C100C100C100C100C100C100C100C100C100C100C100C100C100C100C10180801
:2063D8003804E00300000000000000000000000000000000000000003E7818301810181038
:2063F8001810300830083008300830046004600460046002C002C002C002C00180018001B2
:20641800800080000000000000000000000000000000000000000000CFF38661862184216F
:2064380004210C238C238C238C138C138813481258165816580E380E300E300E300C3004EB
:206458001004100400000000000000000000000000000000000000003E7C181018083008C2
:20647800300460046002C002C0018001800180018003400340062006200E100C100C18183C
:2064980008383E7C00000000000000000000000000000000000000007E7C1C10181018087C
:2064B80030083008300460046004C002C002C001800180018001800180018001800180010B
:2064D8008001E0070000000000000000000000000000000000000000F87F383018300C18F1
:2064F8000418000C000600060003000380018001C000C000600060003000184018600C20DC
:206518000C38FE3F0000000000000000000000000000C03FC000C000C000C000C000C00063
:20653800C000C000C000C000C000C000C000C000C000C000C000C000C000C000C000C00043
:20655800C000C000C000C03F00000000000000000000000000001800180010003000200054
:20657800600060004000C00080008001800100010003000200060006000C000C000C001873
:20659800001800300030003000600000000000000000FC03000300030003000300030003CA
:2065B800000300030003000300030003000300030003000300030003000300030003000393
:2065D800000300030003FC030000000000000000C003C00760041008000000000000000095
:2065F800000000000000000000000000000000000000000000000000000000000000000083
:20661800000000000000000000000000000000000000000000000000000000000000000062
:20663800000000000000000000000000000000000000000000000000000000000000000042
:2066580000000000000000000000FFFF000000007800C000000100000000000000000000EB
:20667800000000000000000000000000000000000000000000000000000000000000000002
:206698000000000000000000000000000000000000000000000000000000000000000000E2
:2066B800000000000000E007180C0C180C180C18001CE01B38180C180618061806180698C8
:2066D8000C9EF87100000000000000000000000000000000000010001E0018001800180019
:2066F8001800180018009807581C38183830183018301830183018301830183018103818FF
:20671800380CC807000000000000000000000000000000000000000000000000000000004E
:20673800000000000000C0077008301818180C180C000C000C000C000C000C20182018109E
:206758003008C0070000000000000000000000000000000000000010001E001800180018AC
:20677800001800180018E01B301C181818180C180C180C180C180C180C180C180818181CC2
:20679800307AE009000000000000000000000000000000000000000000000000000000004E
:2067B800000000000000C003300C101818100C300C300C30FC3F0C000C000C0018201810FF
:2067D8007018C0070000000000000000000000000000000000000000003E80618060C06033
:2067F800C000C000C000FC1FC000C000C000C000C000C000C000C000C000C000C000C00026
:20681800C000F80F0000000000000000000000000000000000000000000000000000000099
:20683800000000000000C077306C10181818181818181018300CF00718001800F803F01F20
:2068580018380C300C300C301818E0070000000000000000000010001E001800180018008F
:206878001800180018009807580C3818181818181818181818181818181818181818181885
:2068980018187E7E00000000000000000000000000000000000000008001C00380010000EF
:2068B800000000000001F801800180018001800180018001800180018001800180018001BA
:2068D8008001F81F0000000000000000000000000000000000000000001C001E000C0000C2
:2068F800000000000008C00F000C000C000C000C000C000C000C000C000C000C000C000C19
:20691800000C000C000C18061802F0010000000000000000000010001E001800180018009C
:20693800180018001800183E180C1804180218019801D801780338031806180C180C181870
:2069580018387E7C0000000000000000000000000000000000000001F80180018001800158
:206978008001800180018001800180018001800180018001800180018001800180018001EF
:206998008001F81F0000000000000000000000000000000000000000000000000000000047
:2069B800000000000400F73C8E6386618661866186618661866186618661866186618661AA
:2069D8008661CFF300000000000000000000000000000000000000000000000000000000F6
:2069F80000000000000090075E0C381818181818181818181818181818181818181818184E
:206A180018187E7E0000000000000000000000000000000000000000000000000000000032
:206A3800000000000000C003300C1018181808300C300C300C300C300C300C3018181818E7
:206A5800300CC003000000000000000000000000000000000000000000000000000000001F
:206A780000000000000090075E0C381818101830183018301830183018301830181838180D
:206A9800780C98071800180018007E000000000000000000000000000000000000000000F5
:206AB800000000000000C013301E181C18180C180C180C180C180C180C180C180818181CE9
:206AD800301EE019001800180018007E000000000000000000000000000000000000000091
:206AF80000000000000060387E666061E001E0006000600060006000600060006000600080
:206B18006000FE0700000000000000000000000000000000000000000000000000000000F8
:206B3800000000000000C02760383030302030207000E003800F001E0038083008301830CE
:206B58003818C80F00000000000000000000000000000000000000000000000080008000F6
:206B78008000C000E000FC1FC000C000C000C000C000C000C000C000C000C000C020C02082
:206B98008011000F000000000000000000000000000000000000000000000000000000003D
:206BB8000000000010101E1E18181818181818181818181818181818181818181818181C1D
:206BD800307AE009000000000000000000000000000000000000000000000000000000000A
:206BF8000000000000003E7C18301810181830083008200460046004C002C002C0038001FF
:206C180080018000000000000000000000000000000000000000000000000000000000005B
:206C3800000000000000DFF3866184218C218C218C13881358135812580E700E300E300C17
:206C58003004200400000000000000000000000000000000000000000000000000000000C4
:206C78000000000000007C3E300870086004C002C00280018001800340062006200C101865
:206C980018183E7E00000000000000000000000000000000000000000000000000000000F0
:206CB8000000000000003E7C18181808100830082004600460044002C002800280018001EE
:206CD80080008000800040007C003C00000000000000000000000000000000000000000024
:206CF800000000000000FC1F0C1C0C0C0406040700038001C001C00060007020302018307F
:206D18000C18FC1F00000000000000000000000000300008000400040004000400040004CC
:206D3800000400040004000400040003800100020004000400040004000400040004000481
:206D58000004000400040008003000000001000100010001000100010001000100010001CD
:206D78000001000100010001000100010001000100010001000100010001000100010001EB
:206D980000010001000100010001000100000000180020004000400040004000400040001D
:206DB800400040004000400040008001000380004000400040004000400040004000400077
:206DD80040004000400020001800000000007800C400824102410027001C0000000000001E
:206DF80000000000000000000000000000000000000000000000000000000000000000007B
:206E1800000000000000000000000000436C656172A1AD0045596F756E6753747564696F56
:206E3800000F0F0F0F0F0F0F0F0F0F0F0F0F0F0F0F5A5A5A5A5A5A5A5A5A5A5A5A5A5A5A04
:206E58005AA5A5A5A5A5A5A5A5A5A5A5A5A5A5101E2C3A48566472808E9CAAB8C6D4E2101A
:1D6E78001E2C3A48566472808E9CAAB8C6D4E2101E2C3A48566472808E9CAAB8C6A3
:06003500E478FFF6D8FD9F
:20001300795CE94400601B7A01906E39780175A000E493F2A308B8000205A0D9F4DAF2758F
:02003300A0FF2C
:1B3FBF0020F71130F6138883A88220F509F6A8837583002280FEF280F5F02201
:0D3FDA00E58330E7076382FF6383FFA322C6
:203FE70074FE2581F8E68582F0A4C0E08582F018E6A4F582D0E025F0C58386F0A42583F5B5
:02400700832212
:20003B007800E84400600A790175A000E4F309D8FC7800E84400600C7900900001E4F0A3C3
:04005B00D8FCD9FAFA
:20400900C02E85812EC082C083E5812406F5817E00E52E24FBF8EE26FAE40836FB08860485
:20402900E52E24FAF8E52E2403F9E6F7097700C006C004C003C002E52E2403F8E6C0E008EF
:20404900E6C0E0A82E088682088683124201AD82AF8315811581D002D003D004D006743005
:204069002DFD8A828B838CF0123FBFC374B98DF063F08095F050158A828B838CF01241E56F
:204089002407FF8A828B838CF0123FBFC006E52E2403F8E6C0E008E6C0E0A82E088682084D
:2040A9008683124283A82E08A68208A68315811581D0060EA82E08E60846600302401AEE11
:2040C90014FFE52E24FBF8EE26FCE40836FD0886068C828D838EF0E4123FBFE52E2408F810
:2040E9007600E52E2408F8C3E664808FF063F08095F05076E52E24FBF8E52E2408F9E72671
:20410900C0E0E40836C0E008E6C0E0E52E2407F8D0E0F618D0E0F618D0E0F6E52E2405F81A
:2041290086820886830886F01241E5FBE52E24FBF8EF26FAE40836FD0886068A828D838E16
:20414900F01241E5FCE52E2405F886820886830886F0EC123FBF8A828D838EF0EB123FBFD6
:20416900E52E2408F8061F0240EB852E81D02E22C02E85812EAE82E583FF30E737E52E241B
:20418900FAF8B60A2FE52E24FBF886030886040886058B828C838DF0742D123FBFE52E24DC
:2041A900FBF874012BF6E43C08F608A605C3E49EFEE49FFFE52E24FAF8E6C0E0E52E24FBF6
:1C41C900F8E6C0E008E6C0E008E6C0E08E828F83124009E58124FCF581D02E22A7
:0D00060075812E1242B4E5826003020003F2
:1C41E50020F71430F6148883A88220F507E6A88375830022E280F7E49322E022E9
:20420100E58124FEF88601188600E84960367A01E825E0F8E933400EF9E58298E58399402E
:20422100030A80ECC3E913F9E813F8C3E58298F5F0E583994005F58385F082C3E913F9E85D
:0542410013F8DAE7228A
:20424600C2D5E58330E70DD2D5E4C39582F582E49583F583E58124FEF8E630E70AB2D518BF
:1D426600E4C396F6E40896F918E6F812428D30D50BE4C39582F582E49583F58322DB
:20428300E58124FEF8E6F918E6F87A10E4FBFCE58225E0F582E58333F583EB33FBEC33FC37
:1142A300EB98F5F0EC994006FCABF0438201DADF229F
:0442B40075820022ED
:00000001FF
